:020000020000FC
:0200000009C035
:1000120055C00CEF0ABB0CEF0BBB07E007BB04E0BB
:1000220008BB0FED0DBF00E808B900E205BF02E012
:1000320000B90FEF01B903E806B900E103B902E024
:1000420000BF02E003BF0EE106BF02E009BF21E0EC
:1000520071E031E044275527662778948895FECFD2
:100062000CEF0BBB04E008BB431708F0C09A531710
:1000720008F0C19A032F0A95E3E4F0E0E00F0027AD
:10008200F01F099406C007C008C009C00AC00BC00F
:100092000CC0DA980895DB980895DC980895DD98ED
:1000A2000895DE980895DF980895C2980895403023
:1000B20009F04A95503009F05A95089515B1062F66
:1000C2000170006807B9369A0027183098F0039536
:1000D2001E3080F00395193168F003951D3250F0FF
:1000E2000395103538F003951F3820F003951E3F15
:1000F20008F00395639560FD04C0401708F4402F93
:1001020003C0501708F4502F2A9549F42EE2A8DFB5
:100112003A9529F437E07A9511F477E0C8DF18951B
:00000001FF
